:020000000130CD
:02000B0021DBF7
:10003000758902D2A9D2AF758C06758A0075816F59
:10004000D2B9D28C7590FF75B0FF75300075310054
:10005000754200C209C20BE52664227025E54164A1
:1000600038701FB210300B2EE5324533453445351C
:1000700054F07010853236853337853438853539FC
:1000800001A2C21075360075370075380175390048
:100090007526227541388536328537338538348563
:1000A0003935C20BC208C20AD2B7753D78753EC851
:1000B000753F0151463009FD317911F2300A0211C4
:1000C000E5200BA130B20201B530080280E775309F
:1000D00000753100754200D208C20AC210C20B512D
:1000E00046C2B780D0C2AF7590FF75B0FF4387029C
:1000F000002230080122D53D0E753D78D53E0875A9
:100100003EC8D53F0280DEA2B3500A753C0E753A58
:1001100001753B0A22D2B7C208C20AD53CF6753C2B
:100120000ED53AF0853B3A153BE53BB40102053B61
:10013000D20B201021E53564097007E5346409709D
:100140000122E5254158753200B43302416275320F
:1001500000B434ED4162E532640170094533453441
:100160004535700122E5254121753200B433024145
:100170002B753200B434ED412B0520C20951957422
:10018000035520F5202432F8E6300E0224109001A9
:10019000BB93300F0274FF43B033F590E52070033A
:1001A000C2B422147006201611C2B52214700620A3
:1001B0001508C2B122201402C2B02214B78C8527C0
:1001C0004544970405FFFFFFFFFFEF10B38881232D
:1001D0004140930001FBFBFBFBFBFFC0E0C0D005EF
:1001E00030740AB530366230D209053174C8B53181
:1001F0002B6231B20C200B24300C210542743CB52B
:10020000421A6242300815E532144534453345350B
:100210007008C208D20AD2B7411C5121D0D0D0E018
:10022000321532E532F4701E7532091533E533F4B8
:1002300070147533051534E534F4700A75340915F6
:1002400035E535F47000752534E535700A752533CC
:10025000E5347003752532220532740AB5322475EF
:10026000320005337406B5331A7533000534740A49
:10027000B534107534000535740AB5350675350981
:10028000753409752534E535700A752533E5347004
:100290000375253222C216C215C214E535700ED27E
:1002A00014E5347008C215E5337002C216E520C2A9
:1002B0000EB40202D20E300808A20C820E920E80FA
:0E02C0000AA20C920FC20F30B30122C20F220D
